:020000040000FA
:02000000A02836
:08000800A000030EA100831209
:0C0010008101210E8300A00E200E0900CB
:10014000203084008001840A80300402031CA2282D
:100150006030AC00AD0083161E3085053330860557
:1001600083128501860107309F00C8308316810005
:100170008312313090007E30920026308316980032
:100180008312803098000C308316990083123D133F
:10019000BD17003083168C00831200308B00810164
:1001A0008E018F010B118B100B108C130C138C1202
:1001B0000C120C118C100C108B173230A9005E2120
:1001C0007A210510BC1A7421BC1A0514A908031D54
:1001D0000514031DA903A201A30186170330A7007C
:1001E0005221A70BF02806170530A7005221A70BB4
:1001F000F62806130310861E0314A40D0530A7006D
:100200005221A70B002986150230A7005221A70B07
:10021000062986110230A7005221A70B0C2986134C
:100220000530A7005221A70B12290730A30006179B
:100230000330A7005221A70B1A2906130310861EAC
:100240000314A40D0330A7005221A70B2429A30BEC
:1002500017292208403E84000008A500240825062E
:10026000A60003194A29BC1B3D29260825050319A8
:100270003B294E2245299021452926082505031DA5
:100280004329A52345290C2345292208403E840003
:10029000250880000830A300A20A2030220203189B
:1002A000DF28172964000F1D08008F018E01B10897
:1002B000031D5C2941240800B1030800BC01051D91
:1002C000BC1785186629051A6629BC16851D6E2976
:1002D000051E6C29BC140800BC150800051E7229F7
:1002E0003C1508003C1408000030BC1B3130AF0046
:1002F000302408003C187F29BD1B080089293D1BBC
:100300000800822967308316990083123D17BD13B8
:1003100008000C308316990083123D13BD170800A6
:100320002208A800A80DA80DA80DF830A8052608D9
:10033000A70027180830A718073027190630A71973
:100340000530271A0430A71A0330271B0230A71BD9
:100350000130A700A8073C1CB8292130AF00302489
:100360002808AF0030242C08B0002030AF00302423
:10037000BC1CE6295430AF0030242808AA005824B9
:100380002C30AF0030246730AF0030242C30AF0069
:1003900030243130AF0030240D30AF0030242C0831
:1003A000B0005430AF0030242808AA0058242C3064
:1003B000AF0030246730AF0030242C30AF00302441
:1003C0003030AF0030240D30AF0030243C1D022A05
:1003D0007830AF0030249030AF0030242808AF00D0
:1003E0003024C030AF0030242C08B0007830AF008B
:1003F00030249030AF0030242808AF003024803003
:10040000AF003024BC1D2D2A5230AF00302488307C
:10041000AA000310A80C03182A150310A80C03182F
:10042000AA142808AF0030242A08AF003024280876
:10043000523A2A06AF0030242C08B0005230AF00E8
:100440003024AA112808AF0030242A08AF00302435
:100450002808523A2A06AF00302401302702031937
:10046000A5170230270203192517033027020319A5
:10047000A516043027020319251605302702031993
:10048000A515063027020319251507302702031981
:10049000A514083027020319251408002208A80013
:1004A000A80DA80DA80DF830A8052608A700271844
:1004B0000830A718073027190630A7190530271A62
:1004C0000430A71A0330271B0230A71B0130A700F6
:1004D000A8073C1C762A2230AF0030242808AF0041
:1004E00030242C08B0002030AF003024BC1CA42ADB
:1004F0005430AF0030242808AA0058242C30AF0014
:1005000030247230AF0030242C30AF003024313032
:10051000AF0030240D30AF0030242C08B000543030
:10052000AF0030242808AA0058242C30AF00302413
:100530007230AF0030242C30AF0030243030AF00A8
:1005400030240D30AF0030243C1DC02A7830AF007D
:1005500030249030AF0030242808AF0030244030E1
:10056000AF0030242C08B0007830AF003024903039
:10057000AF0030242808AF0030240030AF00302412
:10058000BC1DEB2A5230AF0030248930AA00031082
:10059000A80C03182A150310A80C0318AA1428087D
:1005A000AF0030242A08AF0030242808523A2A0627
:1005B000AF0030242C08B0005230AF003024AA1114
:1005C0002808AF0030242A08AF0030242808523A07
:1005D0002A06AF003024013027020319A513023088
:1005E000270203192513033027020319A51204302B
:1005F000270203192512053027020319A511063019
:10060000270203192511073027020319A510083006
:1006100027020319251008002208A800A80DA80D1C
:10062000FC30A80526180730A61806302619053014
:10063000A6190430261A0330A61A0230261B0130F0
:10064000A61B0030AB0003102B0CA700A807A80ABC
:100650002B183D142B1C3D103C1C3C2B3D1C213009
:100660003D182230AF0030242808AF0030242C0879
:10067000B0002030AF003024BC1C562B5430AF00EB
:1006800030242808AA0058242C30AF0030243D1C08
:1006900067303D187230AF0030242C30AF0030246A
:1006A0003130AF0030240D30AF0030243C1D672BBB
:1006B0007830AF0030249030AF0030242808AF00ED
:1006C00030243D1CC0303D184030AF003024BC1DEC
:1006D000842B5230AF0030243D1C88303D188930C7
:1006E000AA000310A80C03182A150310A80C03185D
:1006F000AA142808AF0030242A08AF0030242808A4
:10070000523A2A06AF00302400302B020319A513F9
:1007100001302B020319251302302B020319A512F5
:1007200003302B020319251204302B020319A511E3
:1007300005302B020319251106302B020319A510D1
:1007400007302B020319251008002208A800A80D65
:10075000A80DFC30A80526180730A6180630261963
:100760000530A6190430261A0330A61A0230261BBB
:100770000130A61B0030AB0003102B0CA700A8070C
:10078000A80A2B183D142B1C3D103C1CC72BBC1C6D
:10079000E12B5430AF0030242808AA0058242C3014
:1007A000AF0030243D1C67303D187230AF0030245C
:1007B0002C30AF0030243030AF0030240D30AF008B
:1007C00030243C1DF22B7830AF0030249030AF0045
:1007D00030242808AF0030243D1C80303D18003004
:1007E000AF003024BC1D0F2C5230AF0030243D1C14
:1007F00080303D188130AA000310A80C03182A1578
:100800000310A80C0318AA142808AF0030242A08E3
:10081000AF0030242808523A2A06AF0030240030B6
:100820002B020319A51701302B02031925170230DB
:100830002B020319A51603302B02031925160430C9
:100840002B020319A51505302B02031925150630B7
:100850002B020319A51407302B02031925140800D5
:10086000A908031D080020302E02031808002C08D8
:1008700084002F088000AE0AAC0A6030AC1BAC00CC
:1008800008000C1E0800AE080319080005142D0806
:10089000840000089900AE03AD0A6030AD1BAD00C6
:1008A0002D083002031D08004630B100B0010800D9
:1008B0000A302A02031C722C64302A02031C6F2C9B
:1008C000C8302A02031C6A2CC830AA023230AF009A
:1008D00030246F2C6430AA023130AF0030247624EB
:1008E000AF0030247B24AF0030240800AA13053069
:1008F0008A002A088200AA1705308A002A08820086
:100A000030343034303430343034303430343034C6
:100A100030343034313431343134313431343134B0
:100A2000313431343134313432343234323432349A
:100A30003234323432343234323432343334333484
:100A4000333433343334333433343334333433346E
:100A50003434343434343434343434343434343456
:100A60003434343435343534353435343534353440
:100A7000353435343534353436343634363436342A
:100A80003634363436343634363436343734373414
:100A900037343734373437343734373437343734FE
:100AA00038343834383438343834383438343834E6
:100AB00038343834393439343934393439343934D0
:100AC00039343934393439343034303430343034E2
:100AD00030343034303430343034303431343134F4
:100AE00031343134313431343134313431343134DE
:100AF00032343234323432343234323432343234C6
:100B000030343134323433343434353436343734A9
:100B10003834393430343134323433343434353495
:100B20003634373438343934303431343234333481
:100B3000343435343634373438343934303431346D
:100B40003234333434343534363437343834393459
:100B50003034313432343334343435343634373459
:100B60003834393430343134323433343434353445
:100B70003634373438343934303431343234333431
:100B8000343435343634373438343934303431341D
:100B90003234333434343534363437343834393409
:100BA0003034313432343334343435343634373409
:100BB00038343934303431343234333434343534F5
:100BC00036343734383439343034313432343334E1
:100BD00034343534363437343834393430343134CD
:100BE00032343334343435343634373438343934B9
:100BF00030343134323433343434353436343734B9
:084000000E00010000000100A8
:02400E00543D1F
:00000001FF
